:020000000528D1
:1000080086298B1383120313831203138501860138
:100018008316FF30831603138500FF308600831292
:100028008B138730831681008312C3308312031326
:10003800C100C2018100A0308B00C301FF30C6019E
:10004800C701C800C9000B2983120313C500031098
:10005800430D463E8400831344088000840A450803
:100068008000C30A4308013A0319C3010310430D72
:100078008313463E84000008840A000403193528C7
:10008800801B352800088A00840300088200831634
:1000980003130C128312031335088A0034088200F4
:1000A800831603138C128312031335088A0034084D
:1000B80082008316031398168312031335088A00E7
:1000C8003408820083120313181635088A0034088E
:1000D8008200831203130C081039003A030904390B
:1000E800031D0130B40078288312031336088A00F0
:1000F80035088200831203130C082039003A0309DB
:100108000439031D0130B40089288312031336080B
:100118008A003508820019308316031399001815D0
:1001280018128312031398170030B500A030B400DA
:1001380000308A004B308200003083120313B50070
:10014800AA30B40000308A0054308200063083168A
:100158000313860418138312031318130030B50011
:10016800BA30B40000308A005D308200003083125B
:100178000313B500C430B40000308A006630820032
:10018800831203132C088A002B0882000030831284
:100198000313B600D430B50000308A006D308200F9
:1001A80083120313B4080319DA28DE288312031311
:1001B800AE01CA28831203132D0899002C088A005F
:1001C8002B088200003083120313B600F030B5000C
:1001D80000308A007E30820083120313B4080319AA
:1001E800F628FD28FF3083120313AC00FF30AB0064
:1001F8000529831203131A08AF00AC012F08AB00BE
:100208000529831203132E088A002D08820007305F
:10021800831203139F008316031305100130831202
:100228000313AC001C30AB0000308A008F30820012
:10023800413083120313A600031103192429252929
:100248008029831203130510A20164302202031CC3
:100258002E29392983120313C501FA30C40000007E
:10026800C40B33290000A20A292983120313051499
:100278002608AD000130AC004630AB0000308A00E3
:10028800CA30820083120313A30103302302031C24
:100298004E29652983120313A20164302202031C2C
:1002A8005629612983120313C501FA30C4000000DE
:1002B800C40B5B290000A20A512983120313A30A65
:1002C8004929013083120313AE006F30AD000030AE
:1002D8008A00E6308200831203132C08A5002B083D
:1002E800A4000310A51F031403187B297F29831278
:1002F80003132408A60020298312031321088A0067
:1003080020088200FF00030E8312031383120313D5
:10031800BB00BB0E0A08BC000408BD000B1DA529C4
:10032800410881005030C207B4300318013EFF3A3B
:10033800013EC1000B11FF30C91BA529C807031CCA
:10034800C9077C08BE007D08BF007E08C0004008C1
:10035800FE003F08FD003E08FC003D0884003C0804
:0C0368008A003B088300FF0E7F0E090096
:02400E00103F61
:00000001FF
